:100000000C94340018950000189500001895000015
:10001000189500001895000018950000189500002C
:10002000189500001895000018950000189500001C
:10003000189500000C94ED1018950000189500001C
:1000400018950000189500000C94AE10189500004B
:1000500018950000189500001895000018950000EC
:1000600018950000189500008FEF8DBFC0E8E8E9F3
:100070004E2E84E08EBFD4E0F3E05F2EA89584B7C7
:10008000082E877F84BF88E1992780936000909332
:100090006000EEEFF3E0A0E0B1E088278D933197A8
:1000A000E9F78EE08093C40080E08093C50088E18A
:1000B0008093C100662470E07093B9007AE0709379
:1000C000B8000E9451187091C10070687093C1000F
:1000D000E0E0F0E0A2E0B1E00E94251A0091020108
:1000E000073010F40C94800084E080930201E0E07B
:1000F000F0E0A0E1BB2784E08C937BE70E94141A18
:100100000E943512E1E0F0E0A3E0B1E00E94251A80
:1001100000910301043010F40C949A0081E0809364
:100120000301E1E0F0E0A0E1BB2781E08C937BE7F5
:100130000E94141AE2E0F0E0A5E0B1E00E94251A66
:1001400000910501083010F40C94B20081E0809316
:100150000501E2E0F0E0A0E1BB2781E08C937BE7C2
:100160000E94141AECE5FCE2A5E0B1E08C9199271D
:10017000A4E0B1E00E94CB18E3E0F0E0A6E0B1E03B
:100180000E94251AE4E0F0E0A9E0B1E00E94251AFF
:1001900000910901003110F40C94DA008FE0809393
:1001A0000901E4E0F0E0A0E1BB2781E08C937BE76C
:1001B0000E94141A0E94DD168CE00E942B170E94E8
:1001C000BF168CE00E942B1781E080930B01209AD0
:1001D000529A57985F9A56985E9A549A80E0809304
:1001E000800084E08093810080EB99EB9093850000
:1001F0008093840070916F00716070936F0084E051
:100200008093810081E08093B100239A239A539ACE
:1002100081E28093B0000E94681810E90E94721871
:100220001EEE0E9472180E946A18E1E0F0E00E943F
:10023000D416289A5A9A0E94DA12009103010130CA
:1002400011F00C944B010E94A416E0E2F8E30E9426
:100250009D160E94A416E6E4F8E30E949D160E94F3
:10026000A416ECE6F8E30E949D16A0E8B3E0E6E7EA
:10027000F8E30E94AA180E949516ECE7F8E30E94A2
:100280009D16A0E8B3E0E0E8F8E30E94AA180E94F7
:1002900095160E94A416E2E0F0E00E94D416AEE6A5
:1002A000B1E0ECEEF7E30E94C318A2E7B1E0ECEE98
:1002B000F7E30E94C318A6E7B1E0ECEEF7E30E9473
:1002C000C318AAE7B1E0E0EFF7E30E94C318AEE776
:1002D000B1E0E0EFF7E30E94C318A2E8B1E0E0EF7D
:1002E000F7E30E94C3180E94BF160E94D116E4E9EA
:1002F000F8E30E94B616E1E0F0E00E94D4160E94F6
:10030000BF160E94D116E2EAF8E30E94B6168FE704
:100310001BE00E94CE16ECEAF8E30E94B6168FE7C7
:1003200015E10E94CE16E6EBF8E30E94B6168FE7C1
:100330001FE10E94CE16E0ECF8E30E94B61680E0C2
:1003400080939D0181E080939E0182E080939C01D7
:1003500000919C010E3F18F011F00C94DE010E94F8
:10036000681810919C010E94721862FA16F40C949D
:10037000D4018FEB10919E010E94CE16E8ECF8E3B9
:100380000E94B616A0E8B3E0ECE9F1E00E94E7199C
:100390000E94AE16ADE9B1E08C918F5F8C93AEE90F
:1003A000B1E08C91865F8C930E946A18ACE9B1E051
:1003B0008C918E5F8C9310F40C94A80100919D0198
:1003C000003011F00C94EA010E94BD16EEECF8E347
:1003D0000E94B616E2E0F0E00E94D416789482E81B
:1003E00080931F0183E8809320018FEF97E1AFE9AD
:1003F000B1E08D939C9380E0809321010E941314BF
:1004000088EC9EE1AFE9B1E08D939C9385E0809309
:1004100021010E94131488E880931F0189E88093CA
:1004200020018FEF97E1AFE9B1E08D939C9380E0DD
:10043000809321010E9413148EE49DE1AFE9B1E0A5
:100440008D939C9385E0809321010E94131480E892
:1004500080931F0181E8809320018FEF9FE2AFE935
:10046000B1E08D939C9380E0809321010E9413144E
:1004700086E193E9AFE9B1E08D939C9385E08093A9
:1004800021010E94131428980E94BF165798A6EFC6
:10049000B1E09C9197FF04C04F9B10C09F779C9345
:1004A0004F990CC089E19F9390E00E945F179F9144
:1004B0004F9904C090689C930E94D5145698A6EF5B
:1004C000B1E09C9196FF04C04E9B10C09F7B9C9313
:1004D0004E990CC089E19F9390E00E945F179F9115
:1004E0004E9904C090649C930E940E1580E0809306
:1004F0009A0182E880931F0183E88093200182E0C3
:10050000809321010E94D91393E0AFE9B1E00E94EA
:10051000B018AFE9B1E00D911C910A5F1F4FAFE930
:10052000B1E00D931C93E4EFF7E30E94E91BEFE9C0
:10053000F1E0D190E080FF2400270E94A41A0E94DD
:10054000F41AEDE0F0E0A2E2B1E00E94081A84E0C3
:10055000809321010E94F613A1EAB1E00D911C9154
:1005600002501040A1EAB1E00D931C93E8EFF7E3CD
:100570000E94E91BE1EAF1E0D190E0808FEFE7FE15
:100580008827F82E082F0E94BC1A0E94F41AEDE06A
:10059000F0E0AEE2B1E00E94081AEEE2F1E00E9463
:1005A000701AECEFF7E30E94E91B0E94571A18F04B
:1005B00011F00C94DD020C94E202AAE9B1E08C91F6
:1005C00081608C93EEE2F1E00E94701AEEE6F1E0B9
:1005D0000E94751A0E94571A18F011F00C94F2023A
:1005E0000C94F802EEE2F1E0AEE6B1E00E94081AE7
:1005F000EEE2F1E00E94701AEAE7F1E00E94751A5B
:100600000E94571A10F00C940B03EEE2F1E0AAE7F7
:10061000B1E00E94081AEEE2F1E00E94751AE6E4E9
:10062000F1E00E94701A0E949B1BEDE0F0E0A6E44E
:10063000B1E00E94081AA2E5B1E00D911C910030D2
:1006400050E8150710F00C942B03A2E5B1E00E94CE
:100650003F160C943B03EAE3F1E00E94751AE6E4CE
:10066000F1E00E94701A0E948C1BEDE0F0E0A6E41D
:10067000B1E00E94081AE2E5F1E0D190E080FF24A9
:1006800000270E94A41A0E947A1AE6E4F1E00E9470
:10069000701A0E94F41AEDE0F0E0AAE3B1E00E94C3
:1006A000081AECE6F1E0D190E080FF2400270E94D8
:1006B000A41A0E947A1AE0E6F1E00E94701A0E94E1
:1006C000F41AEDE0F0E0A4E5B1E00E94081AEEE2D1
:1006D000F1E00E94751AE0E6F1E00E94701A0E94B3
:1006E0009B1BEDE0F0E0A0E6B1E00E94081AACE64A
:1006F000B1E00D911C91003050E8150710F00C94FA
:100700008703ACE6B1E00E943F160C949703E4E542
:10071000F1E00E94751AE0E6F1E00E94701A0E9472
:100720008C1BEDE0F0E0A0E6B1E00E94081AECE6D8
:10073000F1E0D190E080FF2400270E94A41A0E94DB
:100740007A1AE0E6F1E00E94701A0E94F41AEDE0D5
:10075000F0E0A4E5B1E00E94081A88E880931F0148
:1007600089E88093200182E0809321010E94D913BF
:1007700093E0AFE9B1E00E94B018AFE9B1E00D91AC
:100780001C910B5F1F4FAFE9B1E00D931C93E4EF99
:10079000F7E30E94E91BEFE9F1E0D190E080FF244C
:1007A00000270E94A41A0E94F41AEDE0F0E0A6E2ED
:1007B000B1E00E94081A84E0809321010E94F613A0
:1007C000A1EAB1E00D911C9102501040A1EAB1E004
:1007D0000D931C93E8EFF7E30E94E91BE1EAF1E0D7
:1007E000D190E0808FEFE7FE8827F82E082F0E9437
:1007F000BC1A0E94F41AEDE0F0E0A2E3B1E00E941E
:10080000081AE2E3F1E00E94701AECEFF7E30E94AD
:10081000E91B0E94571A18F011F00C9411040C9463
:100820001604AAE9B1E08C9182608C93E2E3F1E0D6
:100830000E94701AE2E7F1E00E94751A0E94571AAE
:1008400018F011F00C9426040C942C04E2E3F1E06F
:10085000A2E7B1E00E94081AE2E3F1E00E94701AF8
:10086000EEE7F1E00E94751A0E94571A10F00C94FE
:100870003F04E2E3F1E0AEE7B1E00E94081AE2E3F0
:10088000F1E00E94751AEAE4F1E00E94701A0E94F9
:100890009B1BEDE0F0E0AAE4B1E00E94081AA2E59B
:1008A000B1E00D911C91003050E8150710F40C9444
:1008B0006904EEE3F1E00E94751AEAE4F1E00E94B7
:1008C000701A0E948C1BEDE0F0E0AAE4B1E00E94F7
:1008D000081AE2E5F1E0D190E080FF2400270E94B1
:1008E000A41A0E947A1AEAE4F1E00E94701A0E94A7
:1008F000F41AEDE0F0E0AEE3B1E00E94081AE2E3A2
:10090000F1E00E94751AE4E6F1E00E94701A0E947C
:100910009B1BEDE0F0E0A4E6B1E00E94081AACE613
:10092000B1E00D911C91003050E8150710F40C94C3
:10093000A904E8E5F1E00E94751AE4E6F1E00E94FE
:10094000701A0E948C1BEDE0F0E0A4E6B1E00E947A
:10095000081AECE6F1E0D190E080FF2400270E9425
:10096000A41A0E947A1AE4E6F1E00E94701A0E942A
:10097000F41AEDE0F0E0A8E5B1E00E94081A80E882
:1009800080931F0181E88093200182E08093210100
:100990000E94D91393E0AFE9B1E00E94B018AFE92B
:1009A000B1E00D911C910B5F1F4FAFE9B1E00D93CA
:1009B0001C93E4EFF7E30E94E91BEFE9F1E0D1902B
:1009C000E080FF2400270E94A41A0E94F41AEDE0A0
:1009D000F0E0AAE2B1E00E94081A84E080932101CD
:1009E0000E94F613A1EAB1E00D911C91075010404E
:1009F000A1EAB1E00D931C93E0E0F8E30E94E91B4B
:100A0000E1EAF1E0D190E0808FEFE7FE8827F82E51
:100A1000082F0E94BC1A0E94F41AEDE0F0E0A6E351
:100A2000B1E00E94081AE4E0F8E30E94E91BEAE260
:100A3000F1E00E94701A0E944D1BEDE0F0E0A5EA83
:100A4000B1E00E94081AE5EAF1E00E94751AE6E3B7
:100A5000F1E00E94701A0E948C1BEDE0F0E0A6E32A
:100A6000B1E00E94081AE6E3F1E00E94701AE8E0A3
:100A7000F8E30E94E91B0E94571A18F011F00C9439
:100A800043050C944805AAE9B1E08C9184608C93ED
:100A9000E6E3F1E00E94701AE6E7F1E00E94751AC1
:100AA0000E94571A18F011F00C9458050C945E052A
:100AB000E6E3F1E0A6E7B1E00E94081AE6E3F1E020
:100AC0000E94701AE2E8F1E00E94751A0E94571A1B
:100AD00010F00C947105E6E3F1E0A2E8B1E00E94A9
:100AE000081AE6E3F1E00E94751AEEE4F1E00E94D4
:100AF000701A0E949B1BEDE0F0E0AEE4B1E00E94B2
:100B0000081AA2E5B1E00D911C91003050E81507DC
:100B100010F40C949B05E2E4F1E00E94751AEEE4F7
:100B2000F1E00E94701A0E948C1BEDE0F0E0AEE450
:100B3000B1E00E94081AE2E5F1E0D190E080FF24E4
:100B400000270E94A41A0E947A1AEEE4F1E00E94A3
:100B5000701A0E94F41AEDE0F0E0A2E4B1E00E9405
:100B6000081AE6E3F1E00E94751AE8E6F1E00E9457
:100B7000701A0E949B1BEDE0F0E0A8E6B1E00E9435
:100B8000081AACE6B1E00D911C91003050E8150751
:100B900010F40C94DB05ECE5F1E00E94751AE8E630
:100BA000F1E00E94701A0E948C1BEDE0F0E0A8E6D4
:100BB000B1E00E94081AECE6F1E0D190E080FF2459
:100BC00000270E94A41A0E947A1AE8E6F1E00E9427
:100BD000701A0E94F41AEDE0F0E0ACE5B1E00E947A
:100BE000081A0E942814ADE1B1E00D911C91023C5D
:100BF00051E015070CF002C00C943106ADE1B1E0F4
:100C00000D911C91043F51E015070CF002C00C94AB
:100C10000E06AAE9B1E08C9188608C93ADE1B1E059
:100C20000D911C91015C1140AFE9B1E00D931C9353
:100C3000AFE9B1E00D911C91023350E0150718F0B7
:100C400011F00C942C0600919F0145E0049FA0E157
:100C5000B1E00C920C942F068FEF809310010C944E
:100C6000340680E080931001A0E1B1E08C91809384
:100C7000B40000919201003011F00C94FB06009139
:100C80000A01013011F00C94550680E080930A01AE
:100C90000E94BF165A9B0C9455068FE718E20E94DB
:100CA000CE16EAEEF8E30E94B616A0E8B3E0AF93E2
:100CB000BF93E2E2F1E00E94701A0E946E1711E009
:100CC00002E0BF91AF910E943119E0E8F3E0A0EBA0
:100CD000B1E00E94031A8FE714E00E94CE16A0EB49
:100CE000B1E00E94B016ECEEF8E30E94B616A0E860
:100CF000B3E0AF93BF93E6E2F1E00E94701A0E9466
:100D00006E1711E002E0BF91AF910E943119E0E847
:100D1000F3E0A0EBB1E00E94031A8FE712E10E941A
:100D2000CE16A0EBB1E00E94B016ECEEF8E30E9404
:100D3000B616A0E8B3E0AF93BF93EAE2F1E00E94F9
:100D4000701A0E946E1711E002E0BF91AF910E94ED
:100D50003119E0E8F3E0A0EBB1E00E94031A8FE75D
:100D60001FE10E94CE16EAE2F1E00E94701AECE068
:100D7000F8E30E94E91B0E94571A10F00C94C40675
:100D8000E0EFF8E30E94B616A0EBB1E00E94B016C7
:100D9000ECEEF8E30E94B61682E080930C01EEE2DE
:100DA000F1E0A5EAB1E00E94081A82E080930D010B
:100DB00080E080939E010E943513E2E3F1E0A5EA12
:100DC000B1E00E94081A80E180930D0181E08093D8
:100DD0009E010E943513E6E3F1E0A5EAB1E00E942E
:100DE000081A8EE180930D0182E080939E010E949B
:100DF00035130C94DD0C013011F00C947607009142
:100E00000A01013011F00C94290780E080930A0157
:100E10000E94BF160E94D116E2EFF8E30E94B616B8
:100E20000E94BD16E6EFF8E30E94B6165A9B0C949A
:100E300029078FE718E20E94CE16EAEEF8E30E9437
:100E4000B6168FEB16E20E94CE16EAEFF8E30E9488
:100E5000B61681E080930C0187E080939E01EEE658
:100E6000F1E0A5EAB1E00E94081A85E080930D0147
:100E70000E943513E2E7F1E0A5EAB1E00E94081A0A
:100E800080E180930D010E943513E6E7F1E0A5EAC9
:100E9000B1E00E94081A8BE180930D010E94351386
:100EA00082E080930C01EAE7F1E0A5EAB1E00E945C
:100EB000081A85E080930D010E943513EEE7F1E0FA
:100EC000A5EAB1E00E94081A80E180930D010E941A
:100ED0003513E2E8F1E0A5EAB1E00E94081A8BE1DF
:100EE00080930D010E9435130C94DD0C023011F03B
:100EF0000C94BC0800910A01013011F00C94A40775
:100F000080E080930A010E94BF160E94D116EEEF86
:100F1000F8E30E94B6160E94BD16E2E0F9E30E94D3
:100F2000B6165A9B0C94A4078FE718E20E94CE16BF
:100F3000EAEEF8E30E94B6168FEB16E20E94CE1698
:100F4000EAEFF8E30E94B61681E080930C0187E097
:100F500080939E01EAE3F1E0A5EAB1E00E94081A5D
:100F600085E080930D010E943513EEE3F1E0A5EAE0
:100F7000B1E00E94081A80E180930D010E943513B0
:100F8000E2E4F1E0A5EAB1E00E94081A8BE1809367
:100F90000D010E943513A5E1B1E00D911D912D9138
:100FA0003C91A9EAB1E00D931D932D933C9380E011
:100FB0008093140180E08093130180E080931201FC
:100FC00080E08093110140E851E561E070E0A9EA1A
:100FD000B1E00D911D912D913C910E947E190CF074
:100FE00002C00C940C08A9EAB1E00D911D912D915D
:100FF0003C9140E851E561E070E00E947919A9EA6E
:10100000B1E00D931D932D933D93A4E1B1E08C913C
:101010008F5F8C930C94E30740E15EE060E070E04A
:10102000A9EAB1E00D911D912D913C910E947E198C
:101030000CF002C00C943508A9EAB1E00D911D91A5
:101040002D913C9140E15EE060E070E00E947919F2
:10105000A9EAB1E00D931D932D933D93A3E1B1E077
:101060008C918F5F8C930C940C084CE350E060E003
:1010700070E0A9EAB1E00D911D912D913C910E9483
:101080007E190CF002C00C945E08A9EAB1E00D9143
:101090001D912D913C914CE350E060E070E00E9486
:1010A0007919A9EAB1E00D931D932D933D93A2E127
:1010B000B1E08C918F5F8C930C9435088091A901DD
:1010C00080931101ADEAB1E0E4E1F1E00E94A119E1
:1010D0008FEB14E10E94CE16EDEAF1E0A0E8B3E058
:1010E0001127222702E033270E94E6180E94AE163D
:1010F000ADEAB1E0E3E1F1E00E94A1198FEB18E164
:101100000E94CE16EDEAF1E0A0E8B3E01127222715
:1011100002E033270E94E6180E94AE16ADEAB1E065
:10112000E2E1F1E00E94A1198FEB1CE10E94CE16D2
:10113000EDEAF1E0A0E8B3E01127222702E033272F
:101140000E94E6180E94AE16ADEAB1E0E1E1F1E0DE
:101150000E94A1198FEB10E20E94CE16EDEAF1E099
:10116000A0E8B3E01127222702E033270E94E61807
:101170000E94AE160C94DD0C033011F00C944E0955
:1011800000910A01013011F00C94E60880E0809390
:101190000A010E94BF165A9B0C94E6088FE718E2DA
:1011A0000E94CE16EAEEF8E30E94B6168FEB10E12D
:1011B0000E94CE16E6E2F9E30E94B6168FEB18E223
:1011C0000E94CE16EEE3F9E30E94B61683E0809308
:1011D000210182E880931F0183E8809320010E940F
:1011E000D913ECEFF7E30E94E91BEFE9F1E0D190AE
:1011F000E080FF2400270E94A41A0E94F41AEDE068
:10120000F0E0A5EAB1E00E94081A82E080930D01A7
:101210000E94FB1288E880931F0189E880932001D7
:101220000E94D913ECEFF7E30E94E91BEFE9F1E02C
:10123000D190E080FF2400270E94A41A0E94F41A93
:10124000EDE0F0E0A5EAB1E00E94081A80E18093A9
:101250000D010E94FB1280E880931F0181E88093BA
:1012600020010E94D913E0E1F8E30E94E91BEFE9B5
:10127000F1E0D190E080FF2400270E94A41A0E9490
:10128000F41AEDE0F0E0A5EAB1E00E94081A8EE160
:1012900080930D010E94FB120C94DD0C0A3011F0BA
:1012A0000C94E10900910A01013011F00C948709B6
:1012B00080E080930A010E94BF168CE00E942B17E9
:1012C0000E94D116E0E4F9E30E94B6160E94BD1612
:1012D000EEE4F9E30E94B6168FE716E10E94CE16FF
:1012E000ECE5F9E30E94B6165A9B0C9487098FE748
:1012F00018E20E94CE16EAEEF8E30E94B6168FEBD3
:1013000012E20E94CE16E0E6F9E30E94B616A0EBC8
:10131000B1E0EDE1F1E00E949A19E0EBF1E0A7EB1A
:10132000B1E01127222702E031E00E94E6188FE7A2
:1013300011E10E94CE16AAE9B1E00C9103FB16F46C
:101340000C94A809A7EBB1E00E94B0160C94BB095D
:1013500000919B01003011F00C94B70994E0A0E8D3
:10136000B3E00E9446160E94AE160C94BB09A7EB90
:10137000B1E00E94B016A0EBB1E0E0E1F1E00E9424
:10138000A119A0EBB1E00E942F1AACE9B1E08C9357
:1013900003E040919C01041BADE9B1E00C938FEB9D
:1013A00010E10E94CE1690919D01A0E8B3E00E944A
:1013B00046160E94AE16A0EBB1E00E94B0160C9447
:1013C000DD0C0B3011F00C94020A00910A0101307F
:1013D00011F00C94000A80E080930A010E94BF166D
:1013E0008CE00E942B170E94DA125A9B0C94000A80
:1013F0008FE718E20E94CE16EAEEF8E30E94B616D6
:101400000C94DD0C0C3011F00C94610A00910A016F
:10141000013011F00C94270A80E080930A010E94A9
:10142000BF160E94D116E8E6F9E30E94B6160E94A4
:10143000AD12A2E0B1E08C91A7E9B1E08D938827CD
:101440008C9386E090E0A5E9B1E08D939C930091A8
:101450009901013011F00C945F0A80E080939901AA
:101460008091970180930201EAE2FCE2A2E0B1E000
:101470008C9199270E94CE18A0EBB1E00E94AA1887
:101480000E94BD16A0EBB1E00E94B0168FEB16E0F3
:101490000E94CE16E0E0F0E0A4E1B0E00E94251A40
:1014A00000910201041711F40C945F0AE0E0F0E0EF
:1014B000A2E0B1E07BE70E94141A0E9435120C945E
:1014C000DD0C0D3011F00C94C10A00910A010130BD
:1014D00011F00C94890A80E080930A010E94BF16E3
:1014E0008FE00E942B170E94D116E0E9F9E30E94D9
:1014F000B6160E94AD12A3E0B1E08C91A7E9B1E06D
:101500008D9388278C9383E090E0A5E9B1E08D93DB
:101510009C9300919901013011F00C94BF0A80E076
:10152000809399018091970180930301E6EAFBE2A1
:10153000A3E0B1E08C9199270E94CE18ADECB1E008
:101540000E94AA180E94BD16ADECB1E00E94B01630
:101550008FEB11E00E94CE16E1E0F0E0A4E1B0E0F4
:101560000E94251A00910301041711F40C94BF0A7C
:10157000E1E0F0E0A3E0B1E07BE70E94141A0C94F4
:10158000DD0C0E3011F00C945B0B00910A01013060
:1015900011F00C94E90A80E080930A010E94BF16C2
:1015A0008FE00E942B170E94D116E2EBF9E30E9414
:1015B000B6160E94AD12A5E0B1E08C91A7E9B1E0AA
:1015C0008D9388278C9387E090E0A5E9B1E08D9317
:1015D0009C9300919901013011F00C94590B80E01B
:1015E000809399018091970180930501ECE5FCE2DD
:1015F000A5E0B1E08C919927A4E0B1E00E94CB185E
:101600000E94BD1600910401003011F00C94120BE1
:10161000EEECF9E30E94B6168FEB11E00E94CE16B5
:101620000C94460B00910401013011F00C942A0B2C
:10163000A0E8B3E0E4E0F1E00E94A1190E94AE1638
:10164000EEEDF9E30E94B6168FEB11E00E94CE1684
:101650000C94460BA0E8B3E0E4E0F1E00E94A1198D
:101660000E94AE16ECEEF9E30E94B616009104015A
:101670000A3010F00C94420B8FEB11E00E94CE1652
:101680000C94460B8FEB12E00E94CE16E2E0F0E0E5
:10169000A4E1B0E00E94251A00910501041711F49D
:1016A0000C94590BE2E0F0E0A5E0B1E07BE70E948A
:1016B000141A0C94DD0C009192010F3081E008F4B3
:1016C00080E08F9300919201023181E010F009F0E7
:1016D00080E09F918923882311F40C94DD0C009104
:1016E0000A01013011F00C94390C80E080930A015A
:1016F000009192010F3011F00C94C40B0E94BF16A0
:101700000E94D116EAEFF9E30E94B6160E94BD16B8
:10171000E2E1FAE30E94B616A9E0B1E08C9180FB09
:10172000ACE9B1E0882780F98C930E94C912E8E106
:10173000FAE30E94B616A9E0B1E08C9181FBACE916
:10174000B1E0882780F98C930E94C912E0E2FAE3A5
:101750000E94B616A9E0B1E08C9182FBACE9B1E041
:10176000882780F98C930E94C912EAE2FAE30E946A
:10177000B616A9E0B1E08C9183FBACE9B1E0882713
:1017800080F98C930E94C9125A9B0C94DC0B8FE752
:1017900018E20E94CE16EAEEF8E30E94B6168FEB2E
:1017A00018E20E94CE16E2E3FAE30E94B6168FE03A
:1017B0000E942B170C94EF0B8FE718E20E94CE16B5
:1017C000E0EFF8E30E94B6168FEB18E20E94CE1607
:1017D000E0EFF8E30E94B6168DE00E942B1700910F
:1017E00092010F3011F00C94020CA9E0B1E08C9141
:1017F00080FBA7E9B1E0882780F98D9388278C9337
:101800000C94330C003111F00C94130CA9E0B1E0EE
:101810008C9181FBA7E9B1E0882780F98D93882717
:101820008C930C94330C013111F00C94240CA9E02E
:10183000B1E08C9182FBA7E9B1E0882780F98D9314
:1018400088278C930C94330C023111F00C94330CD8
:10185000A9E0B1E08C9183FBA7E9B1E0882780F98A
:101860008D9388278C9381E090E0A5E9B1E08D937A
:101870009C9300919901013011F00C94DD0C80E0F3
:1018800080939901009192010F3011F00C94660C35
:10189000A7E9B1E08C9180FBA9E0B1E08C9180F9DF
:1018A0008C938FEB15E00E94CE16A9E0B1E08C91ED
:1018B00080FBACE9B1E0882780F98C930E94C912C3
:1018C0008FEB15E00E94CE160C94CA0C003111F07B
:1018D0000C94880CA7E9B1E08C9180FBA9E0B1E001
:1018E0008C9181F98C938FEB1FE00E94CE16A9E0BA
:1018F000B1E08C9181FBACE9B1E0882780F98C9351
:101900000E94C9128FEB1FE00E94CE160C94CA0CE5
:10191000013111F00C94AA0CA7E9B1E08C9180FB85
:10192000A9E0B1E08C9182F98C938FEB1AE10E94CF
:10193000CE16A9E0B1E08C9182FBACE9B1E088273A
:1019400080F98C930E94C9128FEB1AE10E94CE1687
:101950000C94CA0C023111F00C94CA0CA7E9B1E046
:101960008C9180FBA9E0B1E08C9183F98C938FEB93
:1019700013E20E94CE16A9E0B1E08C9183FBACE9A2
:10198000B1E0882780F98C930E94C9128FEB13E293
:101990000E94CE16E4E0F0E0A4E1B0E00E94251A37
:1019A00000910901041711F40C94DD0CE4E0F0E05F
:1019B000A9E0B1E07BE70E94141A00919A0101307E
:1019C00010F40C944B0D0027A5E2B0E08C9180FB45
:1019D00000F9ABE9B1E08C9180FB442740F9041792
:1019E00011F40C94FC0CABE9B1E08C9180FBA5E206
:1019F000B0E08C9180F98C9300910F01003011F0D0
:101A00000C94490D00919A01083010F00C94140DBB
:101A100000919201003011F40C94140D80E0809339
:101A2000920181E080930A0100919A01083010F43C
:101A30000C94260D009192010A3011F40C94260D9D
:101A40008AE08093920181E080930A0100910E0167
:101A5000013010F40C94490D80E080930E01ADE14B
:101A6000B1E00D911C91063252E015070CF002C056
:101A70000C94490D549AE0E0F3E084E690E001977D
:101A80005C9A0E944F175C980E944F17482F492B71
:101A9000B1F70C944F0D289880E080930F010091CE
:101AA0000101013011F00C94F60E289A80E3482FC2
:101AB00000910001041711F00C94630D80E08093F5
:101AC00004010C94E90E81E3482F041711F00C94E3
:101AD0006E0D81E0809304010C94E90E82E3482F9F
:101AE000041711F00C94790D82E0809304010C949A
:101AF000E90E83E3482F041711F00C94840D85E060
:101B0000809304010C94E90E84E3482F041711F02C
:101B10000C948F0D8AE0809304010C94E90E85E308
:101B2000482F041711F00C949A0D8FE08093040154
:101B30000C94E90E86E3482F041711F00C94A50DC0
:101B40008EE1809304010C94E90E87E3482F04177B
:101B500011F00C94B00D8CE3809304010C94E90E09
:101B600083E4482F041711F00C94C80D82E0809391
:101B700003018FE08093090100E010E020E030E0F5
:101B8000A5E1B1E00D931D932D933C930C94E90EC8
:101B900083E5482F041711F00C94690EA6E0B1E01C
:101BA0008C918F5F8C93E3E0F0E0A6E0B1E07BE7FF
:101BB0000E94141AA0EBB1E0E6E0F1E00E94A11946
:101BC000E4E3FAE30E949D16E0EBF1E0A0E8B3E065
:101BD0001127222703E033270E94E6180E9495165A
:101BE0000E94A416E0E4FAE30E949D16A9E0B1E089
:101BF0000C9100FB16F00C940F0EE6E4FAE30E9441
:101C00009D1600910901023010F40C940D0EEAE5C6
:101C1000FAE30E949D160C940F0E0E94A416A9E0F0
:101C2000B1E00C9101FB16F00C94280EECE5FAE300
:101C30000E949D1600910901043010F40C94260EA8
:101C4000EAE5FAE30E949D160C94280E0E94A41661
:101C5000A9E0B1E00C9102FB16F00C94410EE0E714
:101C6000FAE30E949D1600910901083010F40C94CB
:101C70003F0EEAE5FAE30E949D160C94410E0E9485
:101C8000A416A9E0B1E00C9103FB16F00C94540EDD
:101C9000A0EBB1E0EDE1F1E00E949A19E6E8FAE389
:101CA0000E949D160E94A41683E0809303018FE09A
:101CB0008093090100E010E020E030E0A5E1B1E010
:101CC0000D931D932D933C9381E0809307010C9419
:101CD000E90E85E4482F041711F00C94770E80E08C
:101CE0008093070180E0809303010C94E90E84E562
:101CF000482F041711F00C948F0E81E0809303019C
:101D00008FE08093090100E010E020E030E0A5E1E1
:101D1000B1E00D931D932D933C930C94E90E88E450
:101D2000482F041711F00C94E90EEAE9FAE30E9437
:101D30009D160E94A416E4ECFAE30E949D160E94F0
:101D4000A416E2EEFAE30E949D160E94A416E0E0BB
:101D5000FBE30E949D160E94A416E2E2FBE30E94B0
:101D60009D160E94A416E0E4FBE30E949D160E94CB
:101D7000A416EAE5FBE30E949D160E94A416E6E77E
:101D8000FBE30E949D160E94A416EEE8FBE30E946E
:101D90009D160E94A416E8EAFBE30E949D160E948D
:101DA000A416E2ECFBE30E949D160E94A416ECED43
:101DB000FBE30E949D160E94A416E6EFFBE30E943F
:101DC0009D160E94A416E0E1FCE30E949D160E946D
:101DD000A41680E08093010182E2A0E0B1E08C9340
:101DE00081E080930A0181E08093990100910301D1
:101DF000013010F40C94AA104091040100910801E4
:101E0000041710F40C94AA1080E080930801289A1B
:101E100000910301013011F00C947310E0E2F8E33B
:101E20000E949D160E94A416A9E0B1E00C9100FB4F
:101E300016F00C946C0FA0E8B3E0AF93BF93E2E20E
:101E4000F1E00E94701A0E946E1711E002E0BF914B
:101E5000AF910E943119E0E8F3E0A0EBB1E00E94FD
:101E6000031AA0E8B3E0AF93BF93E4E5F1E00E946A
:101E7000701A0E946E1711E002E0BF91AF910E94AC
:101E80003119E0E8F3E0A7EBB1E00E94031AA7EBF9
:101E9000B1E0EAE2FCE30E94351A11F00C94560F0F
:101EA000A7EBB1E0E0E3FCE30E94AA18E6E3FCE361
:101EB0000E949D16A0EBB1E00E949716EEE3FCE3B2
:101EC0000E949D16A7EBB1E00E949716EAE4FCE39E
:101ED0000E949D160E94A416A9E0B1E00C9101FB9E
:101EE00016F00C94C40FA0E8B3E0AF93BF93E6E202
:101EF000F1E00E94701A0E946E1711E002E0BF919B
:101F0000AF910E943119E0E8F3E0A0EBB1E00E944C
:101F1000031AA0E8B3E0AF93BF93E8E5F1E00E94B5
:101F2000701A0E946E1711E002E0BF91AF910E94FB
:101F30003119E0E8F3E0A7EBB1E00E94031AA7EB48
:101F4000B1E0EAE2FCE30E94351A11F00C94AE0F06
:101F5000A7EBB1E0E0E3FCE30E94AA18EEE4FCE3A7
:101F60000E949D16A0EBB1E00E949716E6E5FCE307
:101F70000E949D16A7EBB1E00E949716EAE4FCE3ED
:101F80000E949D160E94A416A9E0B1E00C9102FBEC
:101F900016F00C941C10A0E8B3E0AF93BF93EAE2F4
:101FA000F1E00E94701A0E946E1711E002E0BF91EA
:101FB000AF910E943119E0E8F3E0A0EBB1E00E949C
:101FC000031AA0E8B3E0AF93BF93ECE5F1E00E9401
:101FD000701A0E946E1711E002E0BF91AF910E944B
:101FE0003119E0E8F3E0A7EBB1E00E94031AA7EB98
:101FF000B1E0EAE2FCE30E94351A11F00C940610FD
:10200000A7EBB1E0E0E3FCE30E94AA18E2E6FCE300
:102010000E949D16A0EBB1E00E949716EAE6FCE351
:102020000E949D16A7EBB1E00E949716EAE4FCE33C
:102030000E949D160E94A416A9E0B1E00C9103FB3A
:1020400016F00C944710A0EBB1E0EDE1F1E00E9436
:102050009A19E6E7FCE30E949D16E0EBF1E0A0E8A8
:10206000B3E01127222702E031E00E94E6180E9427
:102070009516EEE7FCE30E949D16A0E8B3E0E0E1D0
:10208000F1E00E94A1190E9495160E94A416A4E5F1
:10209000B1E0E4E1F8E30E94C318A8E5B1E0E4E1AF
:1020A000F8E30E94C318ACE5B1E0E4E1F8E30E9474
:1020B000C318A0E6B1E0E4E1F8E30E94C318A4E687
:1020C000B1E0E4E1F8E30E94C318A8E6B1E0E4E17E
:1020D000F8E30E94C31880E090E0ACE6B1E08D9395
:1020E0009C930C94AA10023011F00C948D10ADEA60
:1020F000B1E0EAE8FCE30E94AA18A0E8B3E0E5E159
:10210000F1E00E9494190E949516EAE8FCE30E940F
:102110009D160E945C110C94AA10033011F00C94CF
:10212000AA1000910701013011F00C94AA1000913F
:102130009A01003011F00C949E10289AADEAB1E09B
:10214000EAE5FAE30E94AA18ECE8FCE30E949D1677
:102150000E945C110C944602F894FFCF0F921F92DC
:102160002F923F924F925F927F92AF92BF920F93C6
:102170001F932F933F934F935F936F937F938F930F
:102180009F93AF93BF93CF93DF93EF93FF938FB75B
:102190008F93A0E0B1E08091C6008C9381E08093A2
:1021A00001018F918FBFFF91EF91DF91CF91BF918F
:1021B000AF919F918F917F916F915F914F913F91DF
:1021C0002F911F910F91BF90AF907F905F904F9094
:1021D0003F902F901F900F9018950F921F922F9263
:1021E0003F924F925F927F92AF92BF920F931F9355
:1021F0002F933F934F935F936F937F938F939F930F
:10220000AF93BF93CF93DF93EF93FF938FB78F93EA
:1022100080EB99EB9093850080938400ABE9B1E06B
:102220008C9180958C9381E080930E0100919B01AD
:10223000003011F00C944011A8E0B1E08C918F5F58
:102240008C93A5E1B1E00E94321600910B010130A0
:1022500010F40C944011ABE0B1E08C918F5F8C9343
:1022600000910B010C3310F40C94401180E080932A
:102270000B015A9881E080930A0181E080939901D3
:102280008F918FBFFF91EF91DF91CF91BF91AF9170
:102290009F918F917F916F915F914F913F912F917E
:1022A0001F910F91BF90AF907F905F904F903F90A4
:1022B0002F901F900F901895A9E0B1E00C9100FBB2
:1022C00016F00C948911A0E8B3E0E2E2F1E00E947C
:1022D000701A0E946E170E949516ADEAB1E00E9436
:1022E0009716A0E8B3E0E4E5F1E00E94701A0E94BE
:1022F0006E170E94951600910901023010F40C949B
:102300008711ADEAB1E00E9497160C9489110E94E2
:10231000A416A9E0B1E00C9101FB16F00C94B611E3
:10232000A0E8B3E0E6E2F1E00E94701A0E946E17A6
:102330000E949516ADEAB1E00E949716A0E8B3E0BE
:10234000E8E5F1E00E94701A0E946E170E9495164F
:1023500000910901043010F40C94B411ADEAB1E01D
:102360000E9497160C94B6110E94A416A9E0B1E041
:102370000C9102FB16F00C94E311A0E8B3E0EAE242
:10238000F1E00E94701A0E946E170E949516ADEA45
:10239000B1E00E949716A0E8B3E0ECE5F1E00E94FE
:1023A000701A0E946E170E9495160091090108305C
:1023B00010F40C94E111ADEAB1E00E9497160C9470
:1023C000E3110E94A416A9E0B1E00C9103FB16F002
:1023D0000C940A12A0EBB1E0EDE1F1E00E949A1931
:1023E000E0EBF1E0A0E8B3E01127222702E031E0C2
:1023F0000E94E6180E949516ADEAB1E00E94971679
:10240000A0E8B3E0E0E1F1E00E94A1190E94951676
:102410000E94A416A4E5B1E0E4E1F8E30E94C31829
:10242000A8E5B1E0E4E1F8E30E94C318ACE5B1E04F
:10243000E4E1F8E30E94C318A0E6B1E0E4E1F8E3C8
:102440000E94C318A4E6B1E0E4E1F8E30E94C318D7
:10245000A8E6B1E0E4E1F8E30E94C31880E090E070
:10246000ACE6B1E08D939C93089500910201003099
:1024700011F00C9448128FEE8093C40080E080939A
:10248000C5007091C0007D7F7093C0000C94AC12A9
:10249000013011F00C94591287E78093C40080E05A
:1024A0008093C5007091C0007D7F7093C0000C9434
:1024B000AC12023011F00C946A128BE38093C400CA
:1024C00080E08093C5007091C0007D7F7093C00054
:1024D0000C94AC12033011F00C947B128DE18093BC
:1024E000C40080E08093C5007091C0007D7F709330
:1024F000C0000C94AC12043011F00C948C128EE0DD
:102500008093C40080E08093C5007091C0007D7FFF
:102510007093C0000C94AC12053011F00C949D1215
:1025200089E08093C40080E08093C5007091C00072
:102530007D7F7093C0000C94AC12063011F00C94A7
:10254000AC1284E08093C40080E08093C500709159
:10255000C0007D7F7093C00008955A9B0C94C512F3
:102560008FE718E20E94CE16EAEEF8E30E94B61654
:102570008FEB18E20E94CE16E2E3FAE30E94B61651
:102580008FE00E942B170C94C8128CE00E942B172E
:10259000089500919C01013011F00C94D512EEE8E1
:1025A000FCE30E94B6160C94D912E2E9FCE30E9407
:1025B000B61608950E94D116E6E4F8E30E94B61616
:1025C0000E94BD16ECE6F8E30E94B616A0E8B3E060
:1025D000E6E7F8E30E94AA180E94AE16E0EFF8E3DF
:1025E0000E94B616A0E8B3E0E0E8F8E30E94AA185B
:1025F0000E94AE160895A0E8B3E0AF93BF93E5EA5A
:10260000F1E00E94701A0E946E1711E002E0BF9183
:10261000AF910E943119E0E8F3E0A0EBB1E00E9435
:10262000031AA0EBB1E00E942F1AACE9B1E08C9341
:1026300006E040919C01041BADE9B1E00C938FE7EB
:1026400010910D010E94CE1690919D01A0E8B3E07B
:102650000E9446160E94AE16A0EBB1E00E94B01692
:10266000E6E9FCE30E94B6160895E5EAF1E00E946F
:10267000701AECEFF7E30E94E91B0E94571A10F45E
:102680000C945A13ECEFF7E30E94E91BE5EAF1E042
:102690000E94701A0E94F41AEDE0F0E0A5EAB1E0A1
:1026A0000E94081AA0EBB1E0EAE9FCE30E94AA1834
:1026B0000C946013A0EBB1E0EAE4FCE30E94AA18DA
:1026C000A0E8B3E0AF93BF93E5EAF1E00E94701A8F
:1026D0000E946E1711E002E0BF91AF910E94311984
:1026E000E0E8F3E0A7EBB1E00E94031AA7EBB1E04A
:1026F000EAE2FCE30E94351A11F00C948513A7EB73
:10270000B1E0E0E3FCE30E94AA18A7EBB1E00E946D
:102710002F1AACE9B1E08C9306E040919C01041BB8
:10272000ADE9B1E00C9390919D01A0ECB1E00E9465
:102730004616E7EBF1E0A0ECB1E00E948E160E9495
:10274000031AE0EBF1E0A0ECB1E00E948E160E94CB
:10275000031A20910C0110910D010E94C416809162
:102760009E01AAE9B1E00E94E0180E94D6180C90E0
:102770000822689409F4E89416F40C94C513A0ECAC
:10278000B1E00E94B0160C94D81300919B01003068
:1027900011F00C94D41396E0A0E8B3E00E94461622
:1027A0000E94AE160C94D813A0ECB1E00E94B016B3
:1027B00008950E94681810911F010E9472181091CC
:1027C00021010E9472180E946818109120010E9435
:1027D00072180E949118A0EAB1E01C930E948F1811
:1027E000AFE9B1E01C930E946A1808950E9468182E
:1027F00010911F010E947218109121010E947218FD
:102800000E946818109120010E9472180E9491186D
:10281000A2EAB1E01C930E948F18A1EAB1E01C93D8
:102820000E946A1808950E94681810911F010E9462
:102830007218109121010E9472181091A0010E943B
:10284000721810919F010E9472180E946A180895D0
:102850000E94681810E90E9472181AEA0E94721801
:102860000E94681811E90E9472180E949118AAE14A
:10287000B1E01C930E948F18A9E1B1E01C930E9463
:102880006A180E94681810E90E94721818EA0E94DB
:1028900072180E94681811E90E9472180E948F181D
:1028A000ACE1B1E01C930E946A180E94681810E91C
:1028B0000E94721819EA0E9472180E94681811E9A1
:1028C0000E9472180E948F18ABE1B1E01C930E9425
:1028D0006A1880911A018093A101A1EAB1E00C91DC
:1028E00007FB16F00C9479148FEF8093A2010C94DF
:1028F0007C1480E08093A201A1EAB1E00D911C91CB
:1029000044E650E00E94A018A1EAB1E00D931C93A8
:10291000A1EAB1E00D911C9109511040A1EAB1E08A
:102920000D931C93ABE1B1E00D911127ACE1B1E047
:102930004D915527041B150BA3EAB1E00D931C9391
:10294000A3EAB1E00D911C9144E650E00E94A0186A
:10295000A3EAB1E00D931C93A3EAB1E00D911C91A1
:10296000ABE1B1E04D9155270E945416A3EAB1E0C6
:102970004D935C93A1EAB1E00D911C91A3EAB1E003
:102980004D915C91040F151FADE1B1E00D931C93C7
:10299000ADE1B1E00D911C914AE050E00E94541667
:1029A000ADE1B1E04D935C93089581E080930A011D
:1029B00081E08093990181E080930F015A990C94F2
:1029C000E7145A9A81E080930B010C940415A2E954
:1029D000B1E08C918F5F8C9300919201043011F0E3
:1029E0000C94F51480E080939201009192010331E0
:1029F00010F40C94FE148AE08093920180E090E041
:102A0000A5E9B1E08D939C9300910B01013010F486
:102A10000C940D1581E080930B01089581E0809363
:102A2000990181E080930F015A990C9420155A9ACC
:102A300081E080930A0181E080930B010C94C91519
:102A4000A5E9B1E00D911C91013050E0150710F49B
:102A50000C944115A7E9B1E00E943F16A7E9B1E047
:102A60004D915C91A5E9B1E00D911C9104171507FA
:102A700010F00C94411580E090E0A7E9B1E08D934F
:102A80009C9300919201013011F00C946D15AEE60B
:102A9000B1E0E8E1F8E30E94C318A2E7B1E0E8E1A1
:102AA000F8E30E94C318A6E7B1E0E8E1F8E30E946A
:102AB000C318AAE7B1E0ECE1F8E30E94C318AEE75F
:102AC000B1E0ECE1F8E30E94C318A2E8B1E0ECE168
:102AD000F8E30E94C3180C94C915023011F00C944D
:102AE000A715AAE3B1E0E4E1F8E30E94C318AEE35E
:102AF000B1E0E4E1F8E30E94C318A2E4B1E0E4E14C
:102B0000F8E30E94C318A6E4B1E0E4E1F8E30E9410
:102B1000C318AAE4B1E0E4E1F8E30E94C318AEE40C
:102B2000B1E0E4E1F8E30E94C31880E090E0A2E5A0
:102B3000B1E08D939C9300E010E020E030E0A5E14F
:102B4000B1E00D931D932D933C930C94C915033064
:102B500011F00C94B3158AE08093920181E0809388
:102B60000A010C94C9150A3011F00C94BF1580E0CD
:102B70008093920181E080930A010C94C9150B3077
:102B800011F00C94C91580E08093920181E080934C
:102B90000A0100910B01013010F40C94D21581E070
:102BA00080930B0108956B65696E652041757367AD
:102BB000616265202020202020202020202020204D
:102BC0002020202020200054657874202020202000
:102BD00020202020202020202020202020202020F5
:102BE00020202020202020004353562028636F6D92
:102BF0006D612073657061726174656429202020A5
:102C00002020202020202020004F70656E466F720B
:102C10006D6174205A65726F20284C6F6756696524
:102C2000772053747564696F290020203234303066
:102C30000020203438303000202039363030002059
:102C400031393230300020333834303000203537DD
:102C500036303000313135323030000000010205AD
:102C60000A0F1E3C0D911D912D913C910F5F1F4F3E
:102C70002F4F3F4F3C932E931E930E930895ED914B
:102C8000FC91EF5FFF4FFC93EE93089580E290304C
:102C900019F08D939A95E9F79C93089509D00E94B5
:102CA000A01800FC10D0089503D01ED001F8F9CF71
:102CB0000024E89457FF02C009D0689400F80BD0B4
:102CC00010F80124089502D009D008955095409538
:102CD0004F5F5F4F0895E89417FF08950095109592
:102CE0000F5F1F4F68940895352F242FE894452BCC
:102CF00011F468940895512F402F0027112780E187
:102D0000440F551F001F111F021B130B416018F4C5
:102D1000020F131F4E7F8A9599F708958F938D9117
:102D20008823E9F711978F910895A0E8B3E08D917A
:102D3000882311F00CD0FBCF08950E94BB18802D82
:102D400011F005D0FACF08958DE001D08AE000900F
:102D5000C00005FEFCCF8093C6000895A0E8B3E054
:102D60008D91882311F071D0FBCF08950E94BB187C
:102D7000802D11F06AD0FACF089580EC6CC081E00C
:102D80006AD018D080E867C08FE7213039F08FEB28
:102D9000223021F08FE8233009F08FEC810F0C9462
:102DA0002B1780E858D0089588EE93E088D03197AB
:102DB000D9F7089583E0992782C08AEF90E00E94B6
:102DC0005F173B9A3A9A399A389A229A219A299807
:102DD00085E090E00E945F172A9843984298419AB4
:102DE000409A2A9AEF93FF93E3EEF0E00E944C178B
:102DF000FF91EF912A9860D02A9AEF93FF93E3EE28
:102E0000F0E00E944C17FF91EF912A9855D02A9A32
:102E1000EF93FF93E3EEF0E00E944C17FF91EF91E8
:102E20002A984AD040982A9AEF93FF93E3EEF0E075
:102E30000E944C17FF91EF912A983ED088E20BD068
:102E40008EE009D086E007D00895299A829505D0B2
:102E500004D032D008952998F9CF859510F4409A7E
:102E600001C04098859510F4419A01C0419885951C
:102E700010F4429A01C04298859510F4439A01C01B
:102E800043982A9AEF93FF93E3EEF0E00E944C17E9
:102E9000FF91EF912A9808953197F1F70895AE2F99
:102EA000BF2F11974A2F4B2BE1F70895689462F8D2
:102EB0000895E89462F8089581E090E000C0EF93EF
:102EC000FF93EE27E82BE92B31F0E0E0F9E03197B2
:102ED000F1F70197D1F7FF91EF9108958DE207FD8A
:102EE0008D938F2D881F802F881F8F57082F6894F0
:102EF000F7F8802F87FF15C080958395082F80E312
:102F00008D938EE28D93802F815228F080E38D93F4
:102F100099279C93089544270A95802F09F196D00C
:102F20001FC0805230F09EE49D9381E48D939D9369
:102F3000EFCF4427DF92EF92FF920F938FE1801B38
:102F400011F0082F83D089D09EE29D930F91FF90BE
:102F5000EF90DF9044270395003209F4D7CF2BD0B0
:102F60003F93ECEEFFE238E12F2D1E2D0D2DFF24B7
:102F7000EE24DD244427000F111F221FA8F42F92F6
:102F80003F920E94BB18102C0E94BB18202C0E945C
:102F9000BB18302C0E94BB183197410DD21CE31C8A
:102FA000F01C3F902F9001C0339631963A9519F757
:102FB0003F9107D0AFCFDD0CEE1CFF1C0A95D9F76F
:102FC0000895002719E058D08F93802B11F00395B6
:102FD00001C08F911A95B9F7802F882309F496CFF5
:102FE0008F91805D8D930A95D9F792CF0065CD1DA5
:102FF00080B2E60E40597307A0ACB90350D6DC018D
:10300000286BEE0094357700CA9A3B0065CD1D0011
:10301000B2E60E0059730700ACB90300D6DC01001C
:103020006BEE0000357700009A3B0000CD1D0000DC
:10303000E60E000073070000B9030000DC01000089
:10304000EE000000770000003B000000F694E794DB
:10305000D79447950A95D1F7089500270DD08F93FF
:1030600003958F2D8E298D29842BC1F78F91805D3B
:103070008D930A95D9F74CCF1F930F93002710E239
:10308000440FDD1CEE1CFF1C001F802F9AE0890BF3
:1030900010F0082F43951A9599F7802F0F911F91E3
:1030A00008953C983D98449A459A089568944093B1
:1030B000BC008F939F9388279927019629F0409110
:1030C000BC0047FFFACFE8949F918F9162F8089572
:1030D00044EAECCF44E94093BC004091BC0044FD7D
:1030E000FCCF08951093BB0044E8E0DF8F939F93DB
:1030F00088279927019671F04091B900487F483F91
:10310000C9F3E894483139F0483229F0403419F0D5
:10311000403509F068949F918F9162F8089544E8D2
:1031200001C044ECC3DF1091BB004091B900487F5F
:10313000483FD9F30895019111912191308108956B
:103140000F92B801469F8001479F100D569F100DAA
:103150000F9008950E94BB180D920020D9F7089592
:10316000903041F00D911C91169507959A95E1F7D5
:103170001C930E930895C89531960020089591E010
:1031800005C092E003C094E001C098E0F4DF0D9226
:103190009A95E1F70895E80FF91FF1CF019601978D
:1031A00021F00E94BB18E9F7FACF089591E0882337
:1031B00021F08894991F8A95E9F7892F90950895B1
:1031C000883018F011968850FBCF08952E2E3F2E90
:1031D000992781918D3209F093958823D1F79A959B
:1031E000E22DF32D112361F0091718F011F0101BD7
:1031F00001C0191B28F021F080E28D931A95E9F7A0
:1032000080818D3219F48D93319604C0222311F000
:103210008BE28D93091738F031F0091B21F080E320
:103220008D930A95E9F781918D938823E1F73323F4
:1032300051F0EA2FFB2F319633958E9182933A9578
:10324000E1F78EE28C93089599278D9193958823C9
:10325000E1F7939511968C9311978E919A95D1F7EA
:103260000895EA2FFB2F00244C918D9103948E3208
:10327000E1F711248D9113948823E1F71A94101625
:1032800040F41197202F2119239580E38D932A95DF
:10329000E9F7113039F59927AE2FBF2FA00DB91FCF
:1032A000A00FB91F8C919C93853308F421C031E0A5
:1032B0008E918E32E9F38D3241F0830F8A3319F407
:1032C00080E331E001C033278C93AE1789F73323B5
:1032D00041F0AE2FBF2FB8DF81E34D3209F43196B4
:1032E000808308958827E00DF81FE00FF81F808382
:1032F0000895041B150B260B370B089504171507AB
:10330000260737070895000F111F221F331F089546
:1033100000951095209530950F5F1F4F2F4F3F4F11
:103320000895019110810FC00E949B180EC00E9449
:103330009B1810C00191108117FF05C03FEF2FEFC0
:1033400004C0008111272227332737FF03C0E0DFA5
:103350008DE28D93CF92DF92EF92AA24BB24CC24EE
:10336000DD24EE2440E2EAE0FF2755E093E380818C
:10337000890F87FD9F7083FD907F891B81935A95EC
:10338000A9F7C1DFAA1CBB1CCC1CDD1CEE1C4A9596
:1033900051F7E894EFE0FF2782910CD0EB30E0F793
:1033A0001EF068948A2D0AD088278D93EF90DF90C5
:1033B000CF900895982F829501D0892F8F70805DCE
:1033C00026F0803309F4089568948D93089541E0C0
:1033D00003C042E001C044E0E40F8827F81F829157
:1033E000982F829506D0892F04D04A95C1F70C9466
:1033F000001A8F708A3008F0895F805D8D93089580
:1034000088278D93089581918D938823E1F70895FE
:1034100094E081918D939A95E1F70895F999FECF03
:10342000E1BDF2BD3196089591E001C092E07B3795
:1034300051F47FB7F894F2DF8D9180BDFA9AF99A32
:103440009A95C9F77FBF7727089591E001C092E070
:10345000E5DFF89A80B58D939A95D1F708958FEFAF
:1034600083959D919923E1F70895689401C0E894AC
:10347000AF93BF938D9116F0919103C00E94BB183A
:10348000902D891718F011F48823A1F7BF91AF91FF
:103490000895B7FE089590E8B91611F4D0FE089586
:1034A0009FEFD91AE90AF90A09F4039508950F92D2
:1034B0008F939F93D216E306F4060FB680E890E848
:1034C000802795270FBE890739F00FB6892B87FD16
:1034D00002C081E008260FBE9F918F910F90089542
:1034E000D190E190F1900191089521913191419114
:1034F00051910895502F2D2D3E2D4F2D612F089560
:10350000D094E094F09491E0D90E9927E91EF91E29
:1035100010950895652F90E8440F551F5927990F6E
:1035200047956078102F90E8FF0C001F0927990F2E
:10353000F794107800380895FF0C90E89027110F49
:103540009795F794092F08951127BD2CDE2CEF2CA9
:10355000F02E0EE1FF2039F4FE2CED2CDB2CBB24E9
:103560000850C2F775C032F00A95BB0CDD1CEE1C8A
:10357000FF1CF9CF8EDFE0CF102FBD2CDE2CEF2CFF
:10358000F02E11234AF4B094D094E094F0949FEF7D
:10359000B91AD90AE90AF90A0EE1FF2039F4FE2C1A
:1035A000ED2CDB2CBB240850C2F752C032F00A9538
:1035B000BB0CDD1CEE1CFF1CF9CF6BDFBDCF2DEC6F
:1035C0003CEC4CEC5DE366270FC08ADF93DFDD2423
:1035D000EE2490E8F92E0FE307C087DF05C022270D
:1035E000332740E251E46627552351F1002381F14E
:1035F00091DF71F11627005850580894050B18F404
:1036000007FD03C025C007FD23C0469537952795C4
:10361000F694E794D79425D0FF202AF0DD0CEE1C19
:10362000FF1C015073F09D2D969548F0DD203AF473
:10363000EE202AF491E0D90E9927E91EF91E7CCFDD
:1036400007C09FE7092FF92A9FEFD92EE92E089589
:10365000DD24EE24FF240027112708950FE79FEFB4
:10366000F2CF9F929924AA24BB2488E1D216E306C4
:10367000F40628F0D21AE30AF40A089401C08894E8
:10368000991CAA1CBB1CDD0CEE1CFF1C8A9571F753
:10369000D92CEA2CFB2C9F9008953CDFD9F05038B0
:1036A000C9F016270058952F90580894091F12F456
:1036B00018F40EC008F00EC00FD0FF202AF0BB0C8B
:1036C000DD1CEE1CFF1C02C0039513F0E2DE34CFBC
:1036D0000C94211B0C94281B9F92FF92EF928D2D2E
:1036E000FF24EE24DD24BB2493E0849F1001829FFD
:1036F000B00CD11CE21CF31C839FD00CE11C2224D3
:10370000F21C9A9531F0BD2CDE2CEF2CFF248F910A
:10371000ECCF9F900895E9DEFDDE503829F090E867
:1037200069270CC00AF045D007CF5FE32227332773
:10373000442701C0DADEEEDE5038B1F3003899F3E9
:10374000902F951B8BF312F434D0FACF983118F0E8
:10375000222733274427983028F0232F342F44275B
:103760009850F9CF992329F04695379527959A9542
:10377000D9F7912F962742F014D0B0F6F794E7943A
:10378000D7940F5F8BF65DCF10D051F008F4B8DE00
:10379000FF2052F2DD0CEE1CFF1C0150CBF751CF85
:1037A00057CFD20EE31EF41E0895D21AE30AF40A8C
:1037B0000895DF92EF92FF920F931F93D22EE32E84
:1037C000F42E052F162F6F915F914F913F912F91FE
:1037D00008950E94BB18202D0E94BB18302D0E9416
:1037E000BB18402D0E94BB18502D089500401CC6E8
:1037F00000401C4600007A430000A04100007A44CB
:103800000000C8426F12833C000096430000204134
:1038100000409C45000000000000C6C200C0794482
:103820002D2D2D2D2D2D2D2D2D2D2D2D2D2D2D2DC8
:103830002D2D2D2D2D2D2D2D2D2D2D2D2D2D2D2DB8
:103840002D2D2D2D00004C4E54203135202D2041A2
:10385000546D65676120333238502C20494E413217
:1038600031392C20445331363231000056657273A1
:10387000696F6E3A2000312E302E31002C2000006E
:1038800032322D31322D323031352032303A32362B
:103890003A3231004932432D427573205363616ED1
:1038A0000000494E413231392D310000494E41323C
:1038B00031392D320000494E413231392D3300006B
:1038C00044533136323100006865783A200049327D
:1038D000432D4572726F722C206E6F20536C61768F
:1038E0006520666F756E64210000C70020560000D9
:1038F00020004D4158004D494E005253540041564E
:10390000470044757263687363686E697474206EEF
:103910006163683A20202064202020682020206DE8
:1039200020202073000053797374656D202F20458B
:10393000696E7374656C6C756E67656E0000C400AB
:1039400054656D706572617475723A20000050574D
:103950004D204C9A667465723A200000B243000014
:10396000486F6D652020C400476573636877696E92
:103970006469676B6569742073657269656C6C65F1
:10398000205363686E6974747374656C6C650000B1
:1039900050726F746F6B6F6C6C2073657269656CBD
:1039A0006C65205363686E6974747374656C6C65C0
:1039B0000000496E74657276616C6C207365726983
:1039C000656C6C65204175736761626500006B6FA3
:1039D0006E74696E756965726C6963680000205366
:1039E000656B756E64652020202020002053656B78
:1039F000756E64656E20202020004B616E846C65BE
:103A00002073657269656C6C6520417573676162CE
:103A1000650055333A20000020202055353A20001B
:103A20002020205532343A200000202020543A2013
:103A30000000C500244E243B4C4E54313520230059
:103A40002443243B0000555F335B562C555D3B49B6
:103A50005F335B6D412C495D00003B00555F355B7A
:103A6000562C555D3B495F355B6D412C495D00002F
:103A7000555F32355B562C555D3B495F32355B6D8A
:103A8000412C495D0000545BB0432C545D3B4661C2
:103A90006E5B50574D2C445D00005F5F5F5F5F5F62
:103AA0005F5F5F5F5F5F5F5F5F5F5F5F5F5F5F5F26
:103AB0005F5F5F5F5F5F5F5F5F5F5F5F5F5F5F5F16
:103AC0005F5F000042656665686C65204C61626FEF
:103AD000726E65747A7465696C204C4E5420313571
:103AE0003A0043202D20537461727420417573672E
:103AF000616265204353562D466F726D61740000FC
:103B000053202D2053746172742041757367616274
:103B100065204F70656E466F726D6174205A6572D4
:103B20006F0054202D2053746172742041757367A7
:103B30006162652054657874666F726D617400000F
:103B400045202D20456E646520417573676162656F
:103B50002073657269656C6C000030202D206B6FDE
:103B60006E74696E756965726C696368652041750C
:103B700073676162650031202D20496E746572762D
:103B8000616C6C20312053656B756E64650032206A
:103B90002D20496E74657276616C6C2032205365FD
:103BA0006B756E64656E000033202D20496E746560
:103BB0007276616C6C20352053656B756E64656E32
:103BC000000034202D20496E74657276616C6C2083
:103BD00031302053656B756E64656E0035202D2085
:103BE000496E74657276616C6C2031352053656B5B
:103BF000756E64656E0036202D20496E7465727690
:103C0000616C6C2033302053656B756E64656E009B
:103C100037202D20496E74657276616C6C203630C9
:103C20002053656B756E64656E002D302E3030004C
:103C3000302E30300000555F333A202000002056EF
:103C4000202020495F333A202000206D4100555F3D
:103C5000353A202000002056202020495F353A20A8
:103C60002000555F32343A200000205620202049A1
:103C70005F32343A200054656D703A20000020B065
:103C800043202050574D3A2020002C002400656925
:0E3C90006E0061757300205700002041200077
:00000001FF
